:020000040800F2
:10000000C80B0024AD020008211A00087B19000863
:10001000B9020008950300081D2700080000000031
:10002000000000000000000000000000251A000889
:100030002104000800000000231A0008D51A000857
:10004000C7020008C7020008C7020008C70200086C
:10005000C7020008C7020008C7020008C70200085C
:10006000C7020008C7020008C7020008C70200084C
:10007000C7020008C7020008C7020008C70200083C
:10008000C7020008C7020008C7020008C70200082C
:10009000C7020008C7020008C7020008C70200081C
:1000A000C7020008C7020008C7020008C70200080C
:1000B000C70200085D1B0008C7020008C70200084D
:1000C000C7020008C7020008C7020008C7020008EC
:1000D000C7020008D9260008C7020008C7020008A6
:1000E000C7020008C702000800000000C70200089D
:1000F000C7020008C7020008C7020008C7020008BC
:10010000C7020008C7020008C7020008C7020008AB
:10011000C7020008C7020008C7020008C70200089B
:10012000C7020008C7020008C7020008C70200088B
:10013000C7020008C7020008C7020008C70200087B
:1001400000000000000000000000000000000000AF
:10015000C7020008C7020008C7020008C70200085B
:10016000C7020008C7020008C7020008C70200084B
:10017000C7020008C7020008C7020008C70200083B
:10018000C7020008C7020008C7020008C70200082B
:10019000C7020008C7020008C7020008C70200081B
:1001A000C7020008C7020008C7020008C70200080B
:1001B000C7020008C7020008C7020008C7020008FB
:1001C000C7020008C7020008C7020008C7020008EB
:1001D000C7020008C7020008C7020008C7020008DB
:1001E000C7020008C7020008C7020008C7020008CB
:1001F000C7020008C7020008C7020008C7020008BB
:10020000C7020008C7020008C7020008C7020008AA
:10021000C7020008C7020008C7020008C70200089A
:10022000C7020008C7020008C7020008000000005B
:10023000C7020008C702000800000000C70200084B
:10024000C7020008C7020008C7020008C70200086A
:10025000C7020008C7020008C7020008C70200085A
:10026000C7020008C7020008C7020008C70200084A
:10027000C7020008C7020008C7020008000000000B
:10028000C702000800000000C702000800000000CC
:1002900000000000C7020008DFF80CD000F068F88A
:1002A00000480047C1270008C80B002406488047C3
:1002B00006480047FEE7FEE7FEE7FEE7FEE7FEE74B
:1002C000FEE7FEE7FEE7FEE7D91A000899020008FC
:1002D0002DE9F05F0546002092469B46884606467B
:1002E000814640241BE0284641464746224600F00E
:1002F0002FF853465A46C01A914110D3114618465A
:10030000224600F016F82D1A67EB01084F462246E8
:100310000120002100F00DF817EB00094E41201ECE
:10032000A4F10104DFDC484631462A464346BDE8D5
:10033000F09F202A04DB203A00FA02F100207047E7
:100340009140C2F1200320FA03F319439040704713
:10035000202A04DB203A21FA02F00021704721FA1A
:1003600002F3D040C2F12002914008431946704781
:10037000064C074D06E0E06840F0010394E80700F2
:1003800098471034AC42F6D3FFF78AFF8C28000858
:10039000AC280008FEE70000F0B5BFF34F8FBFF3B5
:1003A0006F8F1D4900200860BFF34F8FBFF36F8F21
:1003B0001A4C216841F400312160BFF34F8FBFF325
:1003C0006F8F164970310860BFF34F8F081F0068A8
:1003D00043F6FF75104E1036C0F34E31C0F3C9031B
:1003E00005EA4112184642EA80773760401EFAD289
:1003F000491EF5D2BFF34F8F206840F48030206053
:10040000BFF34F8FBFF36F8F03484C30016841F04B
:1004100004010160F0BD000050EF00E014ED00E0C9
:100420007047000010B528B190F83510022903D0AC
:1004300080214165012010BD1D4A4FF4956301687C
:100440008C189C4207D8042280F83520086820F0D8
:100450000100086029E00C6824F00E040C600168BB
:100460000A440A6822F001020A60016E0A6822F456
:1004700080720A6090F85C30012202FA03F10D4BA1
:100480001960D0E919134B60C16E31B10B6823F4C8
:1004900080730B60D0E91C134B60002180F834108E
:1004A00080F83520016D01B18847002010BD0000A3
:1004B000F0FFFDBF045402580248016841F00101F9
:1004C00001607047200400582DE9F84F6C4C002261
:1004D0004FF0B04A4FF0010B4FF0030E4FF00F09F1
:1004E0000B680BFA02F73B40BB4270D14D68022DFE
:1004F00001D0122D12D1D50800EB850CDCF820605C
:100500005507ED0E09FA05F826EA0806D1F810801D
:1005100008FA05F848EA0608CCF82080D0F80080F0
:10052000560091F804C00EFA06F50CF0030C28EA08
:1005300005080CFA06FC4CEA080CC0F800C0D1F81B
:1005400004C0BCF1010F08D0BCF1020F05D0BCF112
:10055000110F02D0BCF1120F16D1D0F808C0D1F89B
:100560000C802CEA050C08FA06F848EA0C08C0F8DA
:100570000880D0F804C02CEA070C0F79C7F30017E5
:10058000974047EA0C074760C768AF438D68B5409E
:100590003D43C5604D68ED006BD53A4D2E6846F081
:1005A00002062E602D6822F0030606F1B04605F023
:1005B00002050095D6F808C495072F0F09FA07F52C
:1005C0002CEA050C304DA84202D100252EE050E067
:1005D0002E4DA84201D1012528E02D4DA84201D180
:1005E000022523E02B4DA84201D103251EE02A4D10
:1005F000A84201D1042519E0284DA84201D10525C2
:1006000014E0274DA84201D106250FE0254DA84250
:1006100001D107250AE0244DA84201D1082505E0B3
:10062000224DA84201D1092500E00A25BD4045EA36
:100630000C05C6F8085425684E689D43F60300D59E
:100640001D43256065684E689D43B60300D51D4374
:100650006560DAF8005056464F689D43FF0200D5AA
:100660001D43356075684F689D43BF0200D51D432B
:100670007560521C102AFFF433AFBDE8F88F0000FC
:1006800080000058F4440258000002580004025848
:1006900000080258000C02580010025800140258BA
:1006A00000180258001C025800200258002402586A
:1006B00042694A40426170470AB1018370474183F1
:1006C0007047000001488068704700001400002453
:1006D0000248816802781144816070471400002448
:1006E000032010B500F058F80F2000F007F808B10B
:1006F000012010BD00F022F8002010BD70B50D4D96
:1007000004464FF47A712878B1FBF0F00A49096881
:10071000B1FBF0F000F086FD48B9102C07D20022A2
:100720002146501E00F018F800206C6070BD0120BA
:1007300070BD00001400002404000024704700284D
:1007400009DB012100F01F0291404009800000F107
:10075000E020C0F8001170470E4BF0B41B68C3F3E3
:100760000223C3F10704042C00D904241D1D072D06
:1007700001D2002300E0DB1E012606FA04F56D1EFF
:100780000D409D409E40761E164045EA0601F0BC95
:1007900001F0C5BF0CED00E0064A00F0070110684B
:1007A0004FF6FF03184040EA012003490843106058
:1007B000704700000CED00E00000FA0510B500F0F5
:1007C0005BFA084909684FF4807292FAA2F201F4C8
:1007D0007061B2FA82F2D140034A515CC8400349C9
:1007E000086010BD18440258642800080400002462
:1007F00010B500F0FBF907490968102292FAA2F23D
:1008000001F07001B2FA82F2D140034A515CC84053
:1008100010BD00002044025864280008364930B555
:100820000A68096812F00302344BC1F305311B68F2
:10083000334C03F010032468DFED320AB7EE001AE0
:10084000C4F3CC0414FB03F300EE103A2E4BB8EEC5
:10085000400A07D02D4C012A01D0022A4AD0B4FB0D
:10086000F1F10BE0244C283C22689506284A03D578
:100870002468C4F3C104E240B2FBF1F101EE901A26
:100880001968B8EE612AC1F3080101EE901A1968DF
:10089000F8EE611A40EE201A31EE810A22EE000ACB
:1008A000C1F34621491C00EE901AF8EE600A80EE72
:1008B000201AFCEEC10AC0ED000A1968C1F3064116
:1008C000491C00EE901AF8EE600A80EE201AFCEE49
:1008D000C10AC0ED010A1968C1F30661491C00EEA6
:1008E000901AF8EE600A80EE201ABCEEC10A80ED84
:1008F000020A30BD074ABFE7284402582C44025878
:100900003C440258000000393844025800093D00B8
:100910000090D00340787D01364930B50A680968F7
:1009200012F00302344BC1F305511B68334C03F43E
:1009300080732468DFED320AB7EE001AC4F3CC04EA
:1009400014FB03F300EE103A2E4BB8EE400A07D02A
:100950002D4C012A01D0022A4AD0B4FBF1F10BE060
:10096000244C283C22689506284A03D52468C4F301
:10097000C104E240B2FBF1F101EE901A1968B8EE41
:10098000612AC1F3080101EE901A1968F8EE611AA4
:1009900040EE201A31EE810A22EE000AC1F3462110
:1009A000491C00EE901AF8EE600A80EE201AFCEE68
:1009B000C10AC0ED000A1968C1F30641491C00EEE6
:1009C000901AF8EE600A80EE201AFCEEC10AC0ED23
:1009D000010A1968C1F30661491C00EE901AF8EE8D
:1009E000600A80EE201ABCEEC10A80ED020A30BD1A
:1009F000074ABFE7284402582C440258444402588E
:100A0000000000394044025800093D000090D00326
:100A100040787D012DE9F047DFF8BC9104460E4691
:100A2000D9F8000000F00700B0420CD2D9F800104D
:100A300021F007013143C9F80010D9F8000000F097
:100A40000700B0427ED12078DFF89081800707D57B
:100A5000D8F80010E26821F00F011143C8F8001027
:100A60002078C00762D0D8F80010A26821F4706125
:100A70001143C8F8001059496068183902281CD081
:100A800003281DD0096801281DD04907002960DA14
:100A9000524F083F396821F0070101433960FFF7E1
:100AA00011FE0546606841F28831022813D0032800
:100AB0001ED001288A4627D034E009688903E5E77B
:100AC00009688901E2E7C905E0E7FFF7FBFD411B83
:100AD000514501D923E08A463868C0F3C200022894
:100AE000F3D123E0FFF7EEFD411B514501D916E09C
:100AF0008A463868C0F3C2000328F3D116E0FFF736
:100B0000E1FD411B51450AD83868C0F3C2000128F5
:100B1000F5D10BE0FFF7D6FD411B514502D903206B
:100B2000BDE8F087386810F0380FF3D1D9F800101D
:100B3000484601F00701B1420DD9016821F00701D3
:100B4000314300E005E00160006800F00700B042BA
:100B500001D00120E4E72078400707D5D8F800103D
:100B6000226921F070011143C8F8001020780107B4
:100B70001B4805D50168626921F0700111430160CD
:100B80002178C90605D50168A26921F4E061114305
:100B900001602078800607D51149091D0868E269BF
:100BA00020F070001043086000F066F8D8F80010DC
:100BB0004FF4807292FAA2F201F47061B2FA82F2FA
:100BC000D140084A515CC840074908600F20FFF730
:100BD00095FD0020A4E700000020005218440258B0
:100BE0001C440258642800080400002410B5FFF7D4
:100BF000E5FD08490968012292FAA2F201F00F010D
:100C0000B2FA82F2D140044A515CC84003490860FC
:100C100010BD000018440258642800080800002491
:100C200010B5FFF7E3FF07490968102292FAA2F214
:100C300001F07001B2FA82F2D140034A515CC8401F
:100C400010BD00001C4402586428000810B5FFF7CE
:100C5000CDFF074909684FF4807292FAA2F201F4BD
:100C6000E061B2FA82F2D140024A515CC84010BD44
:100C70001C440258642800083548F0B50068364D19
:100C800010F03801334809D00411082904D0334E3C
:100C900010290BD018290BD02046F0BD29688906F1
:100CA000FBD52968C1F3C101C840F0BD3046F0BD95
:100CB000274918310A68096812F00302284BC1F36A
:100CC00005111B68274F03F001033F68DFED260A7B
:100CD000B7EE001AC7F3CC0717FB03F300EE103A88
:100CE000224BB8EE400A06D0012A01D0022A2BD0AE
:100CF000B4FBF1F008E02A68920603D52A68C2F333
:100D0000C102D040B0FBF1F001EE900A1868B8EED5
:100D1000612AC0F3080001EE900A1868F8EE611A23
:100D200040EE201A31EE810A22EE000AC0F346207E
:100D3000401C00EE900AF8EE600A80EE201ABCEE2D
:100D4000C10A10EE100AF0BDB6FBF1F0DCE70000BE
:100D5000104402580090D0030044025840787D01AE
:100D60002C440258344402580000003930440258E0
:100D70002DE9F05F04460078DFF8FC8341F2883902
:100D8000DFF8F8A3FE4DC0074ED0D8F8001040465B
:100D9000C1F3C20102291AD00068C0F3C2000328BF
:100DA00005D1DAF8000000F0030002280FD06068D7
:100DB000B0F5803F12D010B1B0F5A02F19D028683F
:100DC00020F480302860286820F4802009E028681A
:100DD000800329D56068002874D025E0286840F495
:100DE00080302860606890B1FFF76CFC06464F4683
:100DF00009E0286840F480202860EFE7FFF762FCF4
:100E0000801BB8427DD828688003F7D50CE0FFF737
:100E100059FC06464F4604E0FFF754FC801BB842DD
:100E2000F0D828688003F7D42078D64F80075AD5A9
:100E3000D8F8001040464FF47C3B11F0380F13D027
:100E40000068C0F3C200032803D1DAF8000080076D
:100E50000AD0E068A8B3296821F01901014329608C
:100E6000FFF730FC06461DE02868400702D5E06821
:100E70000028B1D02868E16820F0190008432860F4
:100E8000FFF720FC064604E0FFF71CFC801B02284D
:100E9000B8D828684007F7D507E0FFF713FC801B98
:100EA0000228AFD828684007F7D538689BFAABF21C
:100EB00020F47C312069B2FA82F29040014339601B
:100EC00011E000E0AEE0286820F001002860FFF7A4
:100ED000F9FB064604E0FFF7F5FB801B022891D8DA
:100EE00028684007F7D42078C00655D5D8F80010F8
:100EF00040464FF0F84BC1F3C201012917D00068FA
:100F000000E0EDE0C0F3C200032805D1DAF80000EC
:100F100000F0030001280AD0E069002828682CD0DE
:100F200040F080002860FFF7CDFB064616E02868F9
:100F3000C00502D5E069802874D138689BFAABF20D
:100F400020F0F841206AB2FA82F290400143396001
:100F500022E0FFF7B7FB801B022899D82868C0055C
:100F6000F7D538689BFAABF2216AB2FA82F220F028
:100F7000F8409140084338600EE020F0800028607F
:100F8000FFF7A0FB064604E0FFF79CFB801B02284E
:100F900087D82868C005F7D42078000724D5774F74
:100FA00060694C37002838680FD040F00100386085
:100FB000FFF788FB064604E0FFF784FB801B02284E
:100FC0008DD838688007F7D50EE020F00100386032
:100FD000FFF778FB064604E0FFF774FB801B02284E
:100FE0007ED838688007F7D42078800623D5A0699A
:100FF000002828680FD040F480502860FFF762FB7B
:10100000064604E0FFF75EFB801B022868D82868CC
:101010008004F7D50FE020F480502860FFF752FBE2
:10102000064605E0D6E0FFF74DFB801B022857D8A7
:1010300028688004F7D42078400744D5524F386898
:1010400040F480703860FFF73DFB064604E0FFF790
:1010500039FB801B642843D83868C005F7D5474F53
:10106000A068483701280AD008B1052811D038688F
:1010700020F001003860386820F0040002E0386891
:1010800040F001003860A06888B1FFF71BFB0646FE
:1010900009E0386840F004003860F0E7FFF712FB21
:1010A000811B49451CD838688007F7D50BE0FFF74E
:1010B00009FB064604E0FFF705FB811B49450FD8F5
:1010C00038688007F7D4606AF0B3D8F80010C1F32D
:1010D000C20103297ED00228286820F0807000E039
:1010E00079E0286003D0FFF7EDFA044687E0FFF7C8
:1010F000E9FA064604E0FFF7E5FA801B02287BD8F0
:1011000028688001F7D4DAF8001040F2F3329143F6
:10111000E26A41EA0211A26A1143CAF8001094F887
:1011200034004FF4FE02218E4002491EA0F50070EB
:1011300080B2C1F308010843218F491E02EA014130
:10114000084394F83C1000E05CE0491E120202EAF9
:10115000016108430949083108600B1D19684FF601
:10116000F872A06C914392FAA2F2B2FA82F2904025
:1011700001431960014809E010440258284402580C
:10118000004402580444025800480258001D0168F7
:10119000226C21F00C01114301600168626C21F0A6
:1011A000020111430160016841F48031016001686E
:1011B00041F400310160016841F48021016001685F
:1011C00041F001010160286840F080702860FFF75D
:1011D00079FA01E018E00FE0044604E0FFF772FA44
:1011E000001B022808D828688001F7D50AE0FFF71D
:1011F00069FA001B022802D90320BDE8F09F286885
:101200008001F4D40020F8E70120F6E74FF0E02158
:101210000428086903D020F004000861704740F0FA
:101220000400FAE7401EB0F1807F10B501D3012021
:1012300010BD4FF0E02460610F21601701F06FFADC
:101240000020A06107202061002010BD704770477A
:10125000704770B50446006801694FF00005C94346
:10126000890715D4C168C943890711D4E91E0161F2
:1012700001202077206880698007204602D0FFF790
:10128000E7FF04E000F0A5F8204600F07BF92577A1
:1012900020680169C943490717D4C168C943490790
:1012A00013D46FF004010161022020772068806967
:1012B00010F4407F204602D0FFF7CAFF04E000F0A0
:1012C00088F8204600F05EF9257720680169C94357
:1012D000090716D4C168C943090712D46FF0080181
:1012E0000161042020772068C0698007204602D071
:1012F000FFF7AEFF04E000F06CF8204600F042F982
:10130000257720680169C943C90617D4C168C94354
:10131000C90613D46FF010010161082020772068FE
:10132000C06910F4407F204602D0FFF791FF04E02F
:1013300000F04FF8204600F025F925772068016974
:10134000C943C90708D1C168C943C90704D1891E67
:101350000161204600F044F9206801696FF08005C2
:10136000C943090607D4C168C943090603D4056106
:101370002046FFF76BFF20680169C943C90507D400
:10138000C168C943090603D405612046FFF75EFF23
:1013900020680169C943490609D4C168C94349069F
:1013A00005D46FF040010161204600F025F9206866
:1013B0000169C94389060BD4C168C943890607D4AA
:1013C0006FF0200101612046BDE87040FFF73FBF8C
:1013D00070BD704770B5044690F83C000D4601287A
:1013E0000ED0012684F83C60022084F83D000C2ACF
:1013F00045D007DC5AB1042A1BD0082A78D12CE04A
:10140000022070BD102A4ED0142A71D15DE02068F0
:1014100000F03AFC2068816941F008018161206890
:10142000816921F004018161206881692A69114381
:1014300011E0206800F076FC2068816941F40061C9
:1014400081612068816921F48061816120688169FE
:101450002A6941EA022181614AE0206800F0AAFC81
:101460002068C16941F00801C1612068C16921F0AB
:101470000401C1612068C1692A69114311E0206833
:1014800000F0DCFC2068C16941F40061C1612068A2
:10149000C16921F48061C1612068C1692A6941EA9A
:1014A0000221C16124E0206800F0FEFC2068416D4B
:1014B00041F0080141652068416D21F0040141655A
:1014C0002068416D2A69114311E0206800F022FD77
:1014D0002068416D41F4006141652068416D21F44F
:1014E000806141652068416D2A6941EA02214165B8
:1014F00084F83D60002084F83C0070BD10B5040005
:1015000003D094F83D0010B107E0012010BD002089
:1015100084F83C00204600F00DF8022084F83D00DD
:101520002068211D00F044FB012084F83D000020CC
:1015300010BD0000114800B587B0016841F00201FC
:101540000160006800F0020005900C48083801684E
:1015500041F0020101600068012100F002000590E5
:1015600002200090CDE901010321CDE903100448D8
:101570006946FEF7A9FF07B000BD0000E844025825
:10158000000402587047000010B5012204460068AC
:1015900000F06EFB0D48216881420BD00C4881425F
:1015A00008D00C48814205D00B48814202D00B483C
:1015B000814203D1486C40F40040486420680188AF
:1015C00041F001010180002010BD00000000014039
:1015D0000004014000400140004401400048014037
:1015E0000349884203D103480221FFF761B87047DD
:1015F000680100240000025870477047704790F857
:10160000791090F87A0008437047000070B50268BE
:101610000446D0691368916810F00F0F64D0594DDB
:1016200003F490760D40354376D0C50707D0DD052D
:1016300005D501251562E26F42F00102E2678207DB
:1016400008D5CA0706D0256802222A62E26F42F056
:101650000402E267420708D5CA0706D025680422BB
:101660002A62E26F42F00202E26702070ED503F03F
:10167000200201F080552A4352EAC17206D0256843
:1016800008222A62E26F42F00802E267E26F002A53
:101690003AD0800608D503F0200001F080510843BD
:1016A00002D0204600F01CFDE06F000703D4206844
:1016B000806840062AD5204600F004FD2068816835
:1016C00049061ED5816821F040018160606FC0B17C
:1016D0002D490165606FFEF7A5FE002814D0606FEC
:1016E000016DBDE870400847850615D503F020055B
:1016F00001F0805635430FD02046BDE8704000F021
:10170000EFBC2046FFF77AFF70BD05E02046FFF7EB
:1017100075FF0020E067F7E7C6024FF020050CD503
:101720004E020AD5E803106284F8795084F87A50A2
:101730002046BDE87040FFF760BF06060AD503F0FB
:10174000800601F400010E4304D02046BDE870403D
:1017500000F056BF41060BD5590609D51168204641
:1017600021F04001116084F8795000F005F9CBE7D1
:101770000002C9D55800C7D5106820F0804010601D
:10178000C2E7000001000010B120000810B50400FD
:1017900003D094F8790010B107E0012010BD0020BB
:1017A00084F87800204600F027F8242084F8790097
:1017B0002068016821F001010160204600F0CCFCA6
:1017C0000128EBD0606B10B1204600F0DFFB2068F1
:1017D000416821F4904141602068816821F02A012C
:1017E00081602068016841F0010101602046BDE888
:1017F000104000F02FBC000010B5006886B01B49F7
:10180000884230D11A48016841F001010160006846
:1018100000F00100059016481030016841F01001F9
:10182000016000680121134C00F0100005904FF496
:10183000007000900220CDE9010103900720694665
:1018400004902046FEF740FE4FF480612046009150
:101850006946FEF739FE2520FEF771FF0322252099
:101860001146FEF779FF06B010BD000000100140E0
:10187000E04402580000025890F87A30202B4CD1F6
:10188000B9B1B2B190F87830012B46D0012380F87D
:1018900078304166A0F86820A0F86A20FF228168AD
:1018A000B1F5805F07D07F2351B1B1F1805F0CD0DB
:1018B00010E001207047016921B940F2FF1107E0F3
:1018C000016909BBA0F86C2004E00169E1B13F2186
:1018D000A0F86C100021C167222280F87A2080F8DD
:1018E000781001688A6842F001028A6001680A681B
:1018F00092000CD50A6842F480720A600068816820
:1019000041F08051816006E0A0F86C30E2E70868A1
:1019100040F490700860002070470220704700007B
:1019200030B50068114988420CD1114A5088010431
:1019300008D411464FF000034404097806D50A295B
:1019400001D0538030BD40F400400DE00D2909D096
:10195000084DC0F30D04401C80B2C72829555080A3
:10196000EFD830BD40F48040508030BD00100140C1
:1019700010000024200000247047FEE7144870B5D2
:1019800086B0016841F004010160016801F00401C2
:101990000591016841F010010160006800260325EF
:1019A000694600F01000059008200124CDE90006EA
:1019B0000848CDE90245FEF787FD20206946CDE9BC
:1019C00000060548CDE90245FEF77EFD06B070BD74
:1019D000E044025800100258000802580E4810B5A2
:1019E00086B0016841F001010160006869460B4C56
:1019F00000F001000590022000900120019002906B
:101A0000032003902046FEF75FFD012220460221BD
:101A1000FEF752FE06B010BDE04402580000025826
:101A2000704770477047000070B5284C9CB025681F
:101A300025F004052560254C00260C34256845F466
:101A400040452560256805F440451B952568AD0493
:101A5000FCD5012400940CAD0396240401940224C7
:101A60000994CDE90A410796082485E80D00CDE9DF
:101A700010466846FFF77CF988B93F201390032091
:101A8000CDE9140640200101CDE91640CDE9180149
:101A900050201A90022113A8FEF7BCFF10B10120BC
:101AA0001CB070BD0A48016841F08001016008481F
:101AB000F430016841F002010160006800F00200AA
:101AC0001B90FEF7F9FC0020EAE700000C480258E2
:101AD00000440258FEF7FCBD1C48016841F4700147
:101AE00001601B49086840F001000860184A0020A6
:101AF000103210600A68174B1A400A60144A1832F4
:101B00001060121D1060121D1060114A2832106002
:101B1000121D1060121D1060121D1060121D106049
:101B2000121D1060121D1060121D10600A6822F450
:101B300080220A6006496031086001200649C1F828
:101B40000801C006014980390860704788ED00E04F
:101B5000004402587FEDF6EA008000510148FFF78B
:101B600078BB000068010024104A10B504460E48F6
:101B7000C2E900010020C2E9020410611046FFF72B
:101B8000BDFC0A4960200C224031086060084860B2
:101B9000022088600548FFF71DFCBDE8104003489F
:101BA0000C21FFF7F1BC0000000400406801002494
:101BB0002DE9F04702884FF0804A254C254D264EEE
:101BC000A042264F264B09D0504507D0A84205D049
:101BD000B04203D0B84201D0984204D122F0700C38
:101BE0004A6842EA0C02DFF87CC0DFF87C80A04241
:101BF000DFF878900FD050450DD0A8420BD0B042FE
:101C000009D0B84207D0984205D0604503D040457E
:101C100001D0484503D122F44075CA682A438D8A11
:101C200022F080022A4302808A68C2620A88028502
:101C3000A04207D0984205D0604503D0404501D06E
:101C4000484501D1098A018601214161BDE8F0873B
:101C5000000001400004004000080040000C00406B
:101C600000040140004001400044014000480140A0
:101C7000012310B5046A8B409C430462036A8A40C6
:101C80001343036210BD00002DE9F043026A22F005
:101C900001020262056A4268836925F002051B4C55
:101CA0001C4E23400C6823F003031B4F1C438B681E
:101CB000DFF868C02B43164DDFF86490A84207D0C8
:101CC000B04205D0B84203D0604501D0484506D1A6
:101CD00023F00808CB6843EA080323F00403A84272
:101CE00007D0B04205D0B84203D0604501D0484586
:101CF00005D14D6922F4407215438A692A43426036
:101D00008461496841630362BDE8F0838FFFFEFF91
:101D10000000014000040140004001400044014037
:101D200000480140F0B5026A22F010020262056A22
:101D300042688369194C1B4E23400C6823F440739E
:101D400043EA042425F020038D6843EA0513144D6B
:101D5000A84201D0B04206D1CF6823F0800343EA05
:101D6000071323F04003A8420AD0B04208D00E4D1A
:101D7000A84205D00D4DA84202D00D4DA84207D172
:101D80004D6922F4406242EA85028D6942EA850289
:101D900042608461496881630362F0BDFF8FFFFE8A
:101DA00000000140000401400040014000440140A7
:101DB00000480140F0B5026A22F480720262026AB1
:101DC0004368C46922F40072184E24F073050C684D
:101DD0002C438D6842EA0522134DA84201D0B0423F
:101DE00006D1CF6822F4006242EA072222F4806220
:101DF000A8420AD0B04208D00D4DA84205D00D4DE2
:101E0000A84202D00C4DA84207D14D6923F440539B
:101E100043EA05138D6943EA05134360C4614968C9
:101E2000C1630262F0BD00000000014000040140F7
:101E300000400140004401400048014030B5026AC2
:101E400022F480520262036A4268C46923F4005398
:101E50000D6824F4E64444EA05248D6843EA05331A
:101E60000C4DA8420BD00C4DA84208D00B4DA842F7
:101E700005D00B4DA84202D00A4DA84204D14D69AD
:101E800022F4804242EA85124260C46149680164DA
:101E9000036230BD000001400004014000400140E9
:101EA000004401400048014030B5026A22F480320B
:101EB0000262046A4268436D24F4003423F0700522
:101EC0000B682B430D8944EA05440D4DA8420BD005
:101ED0000C4DA84208D00C4DA84205D00B4DA8428D
:101EE00002D00B4DA84204D14D6922F4803242EA5F
:101EF00005224260436549688165046230BD000087
:101F00000000014000040140004001400044014045
:101F10000048014030B5026A22F480120262046A6D
:101F20004268436D24F400140D6823F4E04343EA4F
:101F300005230D8944EA05540C4DA8420BD00C4DE5
:101F4000A84208D00B4DA84205D00B4DA84202D0A4
:101F50000A4DA84204D14D6922F4003242EA85229A
:101F6000426043654968C165046230BD00000140BC
:101F7000000401400040014000440140004801408D
:101F800001490860704700004004004090F8341098
:101F9000C90706D001684A68836B22F400321A43ED
:101FA0004A6090F83410890706D501684A68C36B07
:101FB00022F480321A434A6090F83410490706D55B
:101FC00001684A68036C22F480221A434A6090F840
:101FD0003410090706D501684A68436C22F40042B0
:101FE0001A434A6090F83410C90606D501688A6819
:101FF000836C22F480521A438A6090F83410890668
:1020000006D501688A68C36C22F400521A438A60BC
:1020100090F83410490611D501684A68036D22F41E
:1020200080121A434A60016DB1F5801F06D1016824
:102030004A68436D22F4C0021A434A6090F8341093
:10204000090606D501684A68806D22F40022024321
:102050004A607047F8B500250446C567FEF732FBB5
:102060000746206800686FF07E46000708D500220A
:102070003B464FF400112046009600F0FBFA60B991
:102080002068006840070AD500223B464FF48001D3
:102090002046009600F0EEFA08B10320F8BD20209B
:1020A00084F8790084F87A00002084F87850F8BD2C
:1020B00010B5806B0021A0F86A10A0F86210FFF73D
:1020C0009DFA10BD01680A6822F490720A600168E6
:1020D0008A6822F001028A60202180F87A10704715
:1020E00010B5B0F86C2090F87A300168222B05D03A
:1020F000088B40F008000883022010BD898C83689B
:10210000B3F5805F01D103696BB11140426E531C7E
:1021100043661170B0F86A10491E0904090CA0F852
:102120006A1007D015E0436E11401980416E891C7A
:102130004166EFE701680A6822F490720A6001685C
:102140008A6822F001028A60202180F87A10FFF765
:10215000E7FB002010BD00002DE9F04F04460068A9
:102160008025FD4B0021D4F810C087B0A6680F462B
:10217000D4F81C8046EA0C06D4F814C0A26A4CEAD3
:10218000080C46EA0C0632430668DFF8D0C306EABC
:102190000C061643066020684268E66822F4405246
:1021A000324342602268A0699A4201D0266A3043D5
:1021B000A66AB6F1005F04D1D4E90B6C46EA0C06BE
:1021C00030439668DFF898C306EA0C06064396602B
:1021D0002068C26A666A22F00F023243C262E14E90
:1021E0002068E14AB04210D1126802F03802182A81
:1021F00074D005DCCAB3082A7AD0102A47D179E016
:10220000202A7BD0282A7CD17AE0D84EB04209D14E
:10221000126802F00702062A73D2DFE802F053695F
:102220006B6D6F71D24EB04209D1126802F0070295
:10223000062A66D2DFE802F0465C5E606264CD4E3C
:10224000B04209D1126802F00702062A59D2DFE82B
:1022500002F0394F51535557C74EB0420BD1126857
:1022600002F00702062A4CD200E00EE0DFE802F09E
:102270002A4042444648C14EB04209D1126802F099
:102280003802182A38D0BBDCB4E74FF0010538E03B
:10229000BB4EB04209D1126802F00702062A30D2C2
:1022A000DFE802F01026282A2C2EB64EB0420BD1C1
:1022B000126802F00702062A23D2DFE802F00319AF
:1022C0001B1D1F2100251CE098421AD1A64A121D91
:1022D000126802F00702062A13D202E00CE007E0BF
:1022E0000CE0DFE802F0030507090B0D022508E00A
:1022F000042506E0402504E0082502E0102500E062
:102300002025DFF864B2A04E9842DFF880A2ABF13E
:10231000540B73D1102D31D006DC022D09D0042DC1
:102320000AD0082D2FD111E0202D29D0402D2AD1FF
:1023300007E0FEF75DFA13E06846FEF76FFA0198D2
:102340000EE003A8FEF7E8FA049809E0DBF80010B5
:102350005846890610D50068C0F3C1012AFA01F079
:10236000002811D06168894601EB410181420AD8F9
:10237000B0EB093F07D808E05046F3E78448F1E79F
:102380004FF40040EEE7012733E1102D4FF0000835
:102390004ED006DC022D0FD0042D15D0082D04D10F
:1023A0002DE0202D4AD0402D13D00127794AA0F5E9
:1023B0004071914270D9E6E7FEF71AFA626A00238B
:1023C000414636F812200DE06846FEF727FA0198DC
:1023D00003E003A8FEF7A0FA04980023616A36F828
:1023E00011201946FDF774FF62680902030241EAF1
:1023F00010615008181841EB080115E032E0DBF8D5
:1024000000105846890609D500680023C0F3C101B1
:102410002AFA01F0616A36F8112015E0606A00239B
:1024200036F8102050460FE00023FDF751FFBDE7BE
:10243000606A002336F81020554805E0606A0023E2
:1024400036F810204FF400400021FDF741FF09024B
:10245000020241EA10614FEA590010184A4641EB66
:102460000801E1E7E3694FF4004293424DD1082DA2
:1024700023D005DC8DB1012D12D0042D06D112E040
:10248000102D35D0202D3AD0402D11D0012721F02C
:102490000F00C1F3420108435AE0FEF7C1FB16E00A
:1024A000FEF7D4FB13E06846FEF7B8F901980EE09A
:1024B00003A8FEF731FA049809E0DBF8001058464B
:1024C000890608D50068C0F3C1012AFA01F0616AE3
:1024D00036F8111010E0606A36F81010BAFBF1F00F
:1024E0004100606801EB5001B1FBF0F081B2CEE732
:1024F000606A36F810102648B0FBF1F0F0E7606A29
:1025000036F81000B2FBF0F0EAE7082D4AD00ADCFA
:102510000DB3012D43D0042D7FF44DAF6846FEF777
:102520007DF9019809E0102D52D0202D55D0402D75
:10253000F2D103A8FEF7F0F90498616A36F8111099
:10254000B0FBF1F1606801EB5001B1FBF0F080B23B
:102550002168C8604DE01FE0000C0058F369FFCF10
:10256000FFF4FF11001001405444025800440040A1
:1025700000480040004C0040005000400014014062
:1025800000780040007C0040742800080090D003D0
:1025900000093D00FFFC0F00FEF742FBCDE7FEF710
:1025A00055FBCAE7DBF80020594692060AD50968B0
:1025B000C1F3C1022AFA02F1626A36F81220B1FBB5
:1025C000F2F20FE0616A36F81120BAFBF2F209E08C
:1025D000616A36F811200949F1E7616A36F811108D
:1025E000B2FBF1F2616802EB5102B2FBF1F189B288
:1025F000C16007B03846BDE8F08F000000093D001B
:1026000090F87910212901D002207047B0F86210AB
:1026100021B18168B1F5805F13D014E001680A68C8
:10262000920004D58A6822F400028A6003E00A68F6
:1026300022F080020A600068016841F040010160F8
:102640000CE0016961B1C16D4A1CC265026809787C
:102650001185B0F86210491EA0F862100020704782
:10266000C16D02680988C1F308011185C16D891C1B
:10267000C165EEE72DE9F0411E461746884604463F
:10268000069D1CE0681C1AD025B1FEF71BF8801BC4
:10269000A84214D92068016821F4D0710160206833
:1026A000816821F001018160202084F8790084F89C
:1026B0007A00002084F878000320BDE8F0812068CB
:1026C000C16938EA010004D00020B842DAD0002005
:1026D000F3E70120F9E7000070B50D4D00240D4827
:1026E000FEF794FF02E0641CAC4204D80948FEF7F0
:1026F00086FF2028F7D1002402E0641CAC4206D8F3
:10270000054901220348FFF7B7F80028F5D170BD4D
:10271000FFFF0100E800002410000024FEE7090785
:10272000090E002804DB00F1E02080F80014704757
:1027300000F00F0000F1E02080F8141D704702E067
:1027400008C8121F08C1002AFAD17047704700203C
:1027500001E001C1121F002AFBD1704710B50446E9
:102760000420FEF753FD0148046010BD0C00002456
:1027700070B5002405464FF47A7603E0304600F049
:1027800005F8641CAC42F9D370BD000070B54FF081
:10279000E02500216C69094AAB6912685043AA69B7
:1027A0009A42FCD002D2A3EB020302E0A4EB0206A1
:1027B0003344194413468142F1D370BD0C00002408
:1027C000FDF7EAFDFDF78CFF042302220521A0207E
:1027D000FFF72AF94FF4C870FFF7C0FF4FF4E1305C
:1027E00000F024F8FFF7FAF8FFF7C8F8C72140F225
:1027F000F310FFF7B9F90C4C002501264FF496773A
:102800000A20FFF7B5FF20780028608801D0401C1F
:1028100000E0401E608080B2B84200D9257000B947
:102820002670FFF7ADFBEBE7000000240B490A4AD6
:1028300010B5C1E9002000208860C8600861886187
:102840000C2048610846FEF7A1FFBDE8104004498E
:1028500001220248FFF710B800100140E8000024F0
:102860001000002400000000010203040102030420
:1028700006070809010002000400060008000A001B
:102880000C0010002000400080000001AC2800086F
:1028900000000024200000003E270008CC2800088B
:1028A00020000024A80B00004E27000801000000B3
:1028B0000090D0030090D003000000000000000052
:0C28C000010000001000000000000000FB
:040000050800029954
:00000001FF
